:100000000C94A6020C94C3020C94DE020C94C3025E
:100010000C94C3020C94C3020C94C3020C94C3024C
:100020000C94C3020C94C3020C9405220C94C302DA
:100030000C94C3020C94C3020C94C3020C94C3022C
:100040000C94C3020C94C3020C94C3020C94C3021C
:100050000C94C30281068106AD06AD061507400863
:10006000400840083307CC07DD07DD073C003D00B2
:100070003E003F0040004100420043004400450074
:100080003B003A0029000000015122002300240017
:100090002500260027002D002E002A002A0021001E
:1000A00020001F001E00350017001C0018000C0067
:1000B000120013002F00300031005F00150008000F
:1000C0001A0014002B000A000B000D000E000F0098
:1000D00033003400280000005C000900070016000F
:1000E0000400390019000500110010003600370027
:1000F000E5005200380059001B001D001D000000E3
:10010000E10000000000000000000000610060004D
:1001100056005500540000000000000000000000E0
:1001200000002C0000000000E600E7005000510035
:100130004F00620000000000E200E000000000004C
:1001400000000000000000005E005D005B005A003F
:10015000630000000000000000000000010001003A
:100160000100010001000100010001000100010087
:1001700001000100005C000001000100010001001D
:100180000100010001000100010001000100010067
:100190000100010001000100C85CC95CCA5CCB5CC5
:1001A000010001000100010001000100C75CC65C04
:1001B000C45CC35C010001000100010001000100FA
:1001C0000100010001000000010001000100010028
:1001D0000100010001000100010001000100010017
:1001E0000100010001000100010001000100010007
:1001F00001000000000000000000000001000100FC
:1002000001000100010000000000000000000000EB
:1002100000000100000000000100010001000100D9
:1002200001000100000000000100010000000000CA
:1002300000000000000000000100010001000100BA
:1002400001000000000000000000000000047F3FEB
:100250001F643214643214783C1E1E140A052223D3
:10026000252628292A2C2D2F3032333536383A3B93
:100270003D3E4042434547494A4C4E5051535557E5
:10028000595A5C5E6062646668696B6D6F71737504
:1002900077797B7D7F81838587898A8C8E90929404
:1002A00096989A9C9E9FA1A3A5A7A8AAACAEAFB111
:1002B000B3B4B6B8B9BBBCBEBFC1C2C3C5C6C7C95B
:1002C000CACBCCCDCED0D1D2D2D3D4D5D6D7D7D815
:1002D000D9D9DADADBDBDBDCDCDCDCDCDDDDDDDD67
:1002E000DCDCDCDCDCDBDBDBDADAD9D9D8D7D7D66F
:1002F000D5D4D3D2D2D1D0CECDCCCBCAC9C7C6C526
:10030000C3C2C1BFBEBCBBB9B8B6B4B3B1AFAEAC6B
:10031000AAA8A7A5A3A19F9E9C9A98969492908E16
:100320008C8A89878583817F7D7B79777573716FEF
:100330006D6B6968666462605E5C5A5957555351CB
:10034000504E4C4A4947454342403E3D3B3A383681
:10035000353332302F2D2C2A292826252322FFAA97
:100360007F5540000101010101010101010202026A
:100370000202020202020303030303030303040451
:10038000040404040405050505050606060606071B
:100390000707070708080808090909090A0A0A0BD4
:1003A0000B0B0C0C0C0D0D0D0E0E0E0F0F0F101075
:1003B00011111112121313141415151616171718FC
:1003C0001819191A1A1B1B1C1D1D1E1E1F20202167
:1003D0002222232424252626272829292A2B2C2DAE
:1003E0002D2E2F30313232333435363738393A3BCF
:1003F0003C3D3E3F404142434445464748494A4CC4
:100400004D4E4F50515354555658595A5B5D5E5F8F
:10041000616264656668696B6C6D6F707273757725
:10042000787A7B7D7E8082838587888A8C8E8F9187
:10043000939596989A9C9EA0A2A3A5A7A9ABADAFB1
:10044000B1B3B5B7BABCBEC0C2C4C6C9CBCDCFD19B
:10045000D4D6D8DBDDDFE2E4E7E9EBEEF0F3F5F844
:10046000FAFDFF09023B00020100A0FA09040000A6
:1004700001030101000921010100012240000705DB
:1004800081030800010904010001030000000921A3
:100490000101000122320007058303080001120157
:1004A0001001000000085347002000020102000173
:1004B0000A034800420038003500000018034700D6
:1004C0007200610079002000530074007500640020
:1004D00069006F0000000403090405010980A101FF
:1004E000850319012AB700150126B700950175107B
:1004F0008100C0050C0901A101850419012AA0028F
:10050000150126A002950175108100C0050109069C
:10051000A101050719E029E71500250195087501D6
:1005200081029501750881030507190029FF15004F
:1005300026FF009506750881000508190129059513
:100540000575019102950175039103C011241FBE29
:10055000CFE5D8E0DEBFCDBF11E0A0E6B0E0E2EA33
:10056000FCE402C005900D92A432B107D9F723E054
:10057000A4E2B1E001C01D92AE31B207E1F70E94E2
:1005800019140C944F260C940000A82FB92F80E06A
:1005900090E041E050EA609530E009C02D9182275B
:1005A0009795879510F084279527305EC8F36F5F85
:1005B000A8F30895EADF8D939D930895CF93CFB765
:1005C000CF93C395839BE9F7839B0EC0839B0CC09D
:1005D000839B0AC0839B08C0839B06C0C091F50221
:1005E000C395C093F502A6C0DF93C091F402DD2746
:1005F000C450DD4F839B02C0DF91E6CF2F930F9352
:100600001F9300B32FEF03FB20F94F933F9310B3D9
:100610004FEF012703FB21F93BE031C04E7F012F53
:1006200010B3216028C0102F4D7F2260000000B35E
:1006300029C04B7F2460012F000010B32BC010B3E2
:10064000477F28602AC04F7E00B320612CC04F7DB9
:1006500010B320622FC04F7B00B3206432C042270A
:1006600000B349934FEF0000102713FB20F910B39C
:100670001C70C9F1297F91F2012703FB21F900B316
:10068000237F89F2315058F1102713FB22F910B360
:10069000277E79F2012703FB23F92F7C81F200B337
:1006A000102713FB24F92F7971F200C010B3012732
:1006B00003FB25F92F7359F200C000B3102713FB79
:1006C00026F9223040F200C010B3012703FB27F9BE
:1006D000243028F64F77206810B30000F9CF10E8D7
:1006E0001ABF00271CC03B503195C31BD04010E8F7
:1006F0001ABF0881033C11F10B3401F12091F10282
:100700001981110F1213EDCF4A81441F093669F187
:100710000D3211F0013E29F74F7009F0042F0093BC
:10072000FA023F914F911F910F912F91DF91CAB71C
:10073000C7FD47CFCF91CFBFCF9118952091FA0237
:10074000222379F31091F802112309F044C03430C8
:100750000AF443C03093F8022093F3021091F4029C
:100760003BE0311B3093F40238C00091F8020130B5
:1007700094F50AE54F7049F43091840034FD2FC0A0
:1007800000938400CEECD2E02EC0433059F04430C8
:1007900091F03091D90234FD22C00093D902CAED04
:1007A000D2E021C03091120334FD19C0009312032E
:1007B000C3E1D3E018C03091E50234FD10C00093CE
:1007C000E502C6EED2E00FC02795A8F45150A9F477
:1007D000220F0000F9CF4AE503C042ED01C0432FCC
:1007E000C4E1D0E032E011B31C60939A11BB02B3B4
:1007F00020E41CE05F93012756E002BB279520F41C
:10080000515021F4220FF9CF012756E000003B5A46
:1008100002BBD0F2279528F4515029F4220F000092
:10082000F9CF012756E0279502BB20F4515021F45F
:10083000220FF9CF012756E02991332302BB21F67D
:10084000037F1091F902110FC651D04002BB11F085
:100850001093F10210E81ABF086011B3137F402F04
:10086000437F5F9100C000C002BB11BB42BB59CFA8
:1008700081E0089581E008950C943A0408950C9461
:100880003E041F93CF93DF9300D000D01F92CDB7CB
:10089000DEB749835A836B833091270189819A811E
:1008A000311114C0662359F0222349F00E94790ABD
:1008B000182F682F89819A810E94220A03C00E9402
:1008C0004D0A182F69817A81812F04C00E94790A0C
:1008D00069817A810F900F900F900F900F90DF91A8
:1008E000CF911F910C94A111FC01262F40815181C1
:1008F0006281738184810C94410481E00895CF93D7
:10090000DF93EC0160E00E947404BE01DF91CF919F
:100910000C943F040C94D0120C94CC1208950E94B5
:10092000CC080E948E042FEB87E299E02150804092
:100930009040E1F700C000000C942B220F931F930E
:10094000CF93DF938C0161E00E947404EC01B80145
:100950000E943C04882309F44BC0B801CE010E94D8
:10096000141C882309F444C0B801CE010E94E71F7B
:100970008823F1F1B801CE010E94131D8823C1F133
:10098000B801CE010E94431F882391F1B801CE0126
:100990000E94581A882361F1F8018281882309F1A5
:1009A000CB358DE5D807C1F050F4C115FCE5DF0764
:1009B00081F0CF3DDC45A9F40E94AA0F19C0CC35C7
:1009C000EDE5DE0761F0CD35DD4559F40E94F30E0B
:1009D00008C00E948F040CC00E94FC0E02C00E943E
:1009E000FF0EC801DF91CF911F910F910C94380435
:1009F00080E0DF91CF911F910F9108950E94AF2168
:100A000080E00E94491C0C9437050E94381B0E940C
:100A10003A050C94B52108950C940B0581E00895D6
:100A2000CF93C82F0E940E05882379F0C0FF02C023
:100A3000909A01C09098C1FF02C0919A01C091980C
:100A4000C2FF02C0969A01C09698CF910895889AE5
:100A50009098899A91988E9A96980895CF93C82FD6
:100A60000E940C058C2F0E941005CF91089580E004
:100A70000C942E050E941C210C942E050E941C2112
:100A800090912601891721F0809326010C942E0560
:100A90000895CF93DF93CDB7DEB72B970FB6F894B9
:100AA000DEBF0FBECDBF4F83588769877A878B879C
:100AB00061110E943F0E9E012F5F3F4F86E0F901BA
:100AC00011928A95E9F785E0FE013796D9010190E8
:100AD0000D928A95E1F789819A814C815D81452B40
:100AE00031F09F3F31F491E08F3F19F403C091E062
:100AF00001C090E090FF09C049815A816B817C81DF
:100B00008D819E810E94600D05C0C9010E947D04F7
:100B10008111F2CF2B960FB6F894DEBF0FBECDBF7A
:100B2000DF91CF910895FC01808191810E94BB0AE1
:100B30000895CF93882309F44DC0C82F8CEF8C0FF4
:100B4000813AF8F48C2F0E94071F811143C06C2F4B
:100B500080916200909163000E946B21882349F08C
:100B60006C2F80916200909163000E94A3210E94EB
:100B7000610E6C2F80916200909163000E94A12110
:100B80000CC080E28C0F883058F4C77081E001C03F
:100B9000880FCA95EAF70E94220ECF910C94610E3D
:100BA000EBE5EC0FE33040F4F0E0ED54FF4F8081D3
:100BB00090E0CF910C943321C85AC73158F4EC2FF0
:100BC000F0E0EE0FFF1FEB57FF4F80819181CF9137
:100BD0000C944921CF910895882349F1682F8CEF17
:100BE000860F813A38F480916200909163000E94F0
:100BF000A3210CC080E2860F883050F4677081E03A
:100C000001C0880F6A95EAF70E94280E0C94610EC5
:100C10008BE5860F833020F480E090E00C94332144
:100C2000685A673120F480E090E00C9449210895DF
:100C30001F93CF93DF93182FEB010E949905209704
:100C400041F087EB9BE00197F1F700C0000021978E
:100C5000F6CF812FDF91CF911F910C94EC05893352
:100C600019F060E070E002C060E570E00C941806D6
:100C7000882321F00E94220E0C94610E089588238F
:100C800021F00E94280E0C94610E0895CF92DF92FD
:100C9000EF92FF920F931F93CF93DF937C01D62F98
:100CA000C72FFC011281058102950F700E94180E5A
:100CB0008823B9F01123A9F08C2F807F803421F094
:100CC00080E28D0F883068F08091940282FD09C027
:100CD00082E00E94C10E0E94180E91E0D82ED92603
:100CE00001C0D12CCC2EC2948FE0C8228C2D90E074
:100CF0008C30910508F0C4C1FC01E65DFF4F0C94F7
:100D00009E258C2F807FCF70882311F0C295C07FE5
:100D1000112399F0CC2309F49FC180E28D0F883014
:100D200010F0D11104C08C2F0E94220E03C08C2F12
:100D30000E94320E0E94610E8FC18D2F0E94EC0521
:100D4000CC2309F49DC180E28D0F883038F1DD237A
:100D500029F18C2F0E94380E24C08C2F807FCF70F9
:100D6000803211F0C295C07FDD2319F0D130A1F19E
:100D70003DC08091940282FF17C0112349F0CC231B
:100D800029F08C2F0E94220E0E94610E80E065C126
:100D900080E00E94EC05CC2309F472C18C2F0E94E4
:100DA000280E0E94610E6CC1112371F0002341F0E6
:100DB000013031F40E94420E8C2B0E944A0E60C119
:100DC0000E94420E8C2B1DC0002319F0013009F443
:100DD00057C10E94570E25C0112321F0063008F09C
:100DE0004FC10EC0053008F04BC11BC0112361F08C
:100DF000002331F0F701858180FF2EC18F7085833C
:100E00008C2F0E9438063CC1002359F0D93309F0D9
:100E100034C1FFEF0DEE12E0F15000401040E1F759
:100E20002AC18C2F0E943F062BC18C2F8695869558
:100E3000837019F0813061F023C1112321F08D2FCF
:100E40009C2F937002C080E090E00E94332120C16B
:100E5000112321F08D2F9C2F937002C080E090E031
:100E60000E94492115C18C2F837009F047C01111D0
:100E70000BC12D2F229526952770220F220F6D2F43
:100E80006F70862F90E0A0E0B0E0022E04C0880FC3
:100E9000991FAA1FBB1F0A94D2F7D4FF10C04FE0BE
:100EA00050E060E070E004C0440F551F661F771FDC
:100EB0002A95D2F7409550956095709503C040E013
:100EC00050E0BA01C695C695C3708A019B01082BF4
:100ED000192B2A2B3B2BC901B801C23049F058F419
:100EE000C13019F00E943809CFC00E942609CCC039
:100EF0000E944A09C9C00E942409C6C0112319F0E2
:100F00008C2F817001C08695882309F4BDC02D2FD8
:100F1000229526952770220F220F6D2F6F70862F36
:100F200090E0A0E0B0E0022E04C0880F991FAA1F35
:100F3000BB1F0A94D2F7D4FF10C04FE050E060E02E
:100F400070E004C0440F551F661F771F2A95D2F723
:100F5000409550956095709503C040E050E0BA010F
:100F6000C695C695C3708A019B01082B192B2A2BA5
:100F70003B2BC901B801C23049F058F4C13019F017
:100F80000E94FD0981C00E94EB097EC00E940F0AE9
:100F90007BC00E945E0978C0CF70112339F08C2F7E
:100FA0000E9484098D2F0E9438066EC08D2F0E94EA
:100FB0003F068C2F0E94A50967C0D23F21F128F47B
:100FC000D03F41F0D13FC1F043C0D33F19F1D43FEE
:100FD00079F03EC0112341F0053008F051C08C2F4C
:100FE0008F710E94CA094CC0063008F049C0F7CF83
:100FF0008091940282FF18C0112339F08C2F8F71D9
:101000000E9484093DC01123C9F38C2F8F710E9467
:10101000A50936C0112329F08C2F8F710E946F090A
:101020002FC00E946A092CC0112349F0CF718C2F68
:101030000E94840963E08C2F0E94A60E21C081E0EB
:101040000E94C10E0230E0F082E00E94C10E18C082
:10105000112331F0002391F28D2F0E94990510C0C9
:10106000002399F2D93349F41FEF2DEE32E01150ED
:1010700020403040E1F700C000008D2F0E94EC05B9
:1010800088EF8C0D843020F40E941C210E942E05D4
:10109000DD20C9F00E94140E80FD15C0F7011282F8
:1010A0000E940E0E0E948409C7010E9484080E94BB
:1010B0000E0EDF91CF911F910F91FF90EF90DF9077
:1010C000CF900C94A509DF91CF911F910F91FF90C4
:1010D000EF90DF90CF9008950F931F93CF93DF93FE
:1010E000EC01688179818A810E94C60A8C010E9484
:1010F000210A0E941209B801CE010E944606DF9122
:10110000CF911F910F910895CF93DF93EC019881B8
:1011100089812B813C81232B31F08F3F31F481E099
:101120009F3F19F403C081E001C080E080FD1DC035
:10113000CE010E949E04811110C00E94180E8823C7
:10114000A1F08A81882389F08091940282FD0DC0EC
:1011500082E0DF91CF910C94C10ECE010E946C0809
:10116000CE01DF91CF910C947F04DF91CF91089550
:1011700080E090E00E94332180E090E00E944921CD
:101180000E943F0E0C94610E80916200909163006A
:101190000E94A5210C94B8080E942F0E0C94C4083C
:1011A00092959F70963079F010F4925001C09A5049
:1011B000923068F4803F69F018F4883E40F409C02A
:1011C000843F29F406C0883E20F0813F11F080E082
:1011D000089581E00895FC01808191810E94BB0AFD
:1011E0000E94D0080895CF93DF9300D000D01F92C3
:1011F000CDB7DEB70F900F900F900F900F90DF914B
:10120000CF910895CF93DF9300D000D000D0CDB719
:10121000DEB726960FB6F894DEBF0FBECDBFDF91C6
:10122000CF910895089508950C9413090C9414090E
:101230000E94160960937701709378018093790179
:1012400090937A010C94B8080C9418090F931F938B
:1012500000917701109178012091790130917A0104
:10126000602B712B822B932B1F910F910C941809DB
:101270000F931F93009177011091780120917901CC
:1012800030917A0160237123822393231F910F9160
:101290000C9418090F931F93009177011091780116
:1012A0002091790130917A01602771278227932755
:1012B0001F910F910C9418090C9413090E945C095A
:1012C000609373017093740180937501909376011C
:1012D0000C94B80860E070E0CB010C945E090F93A9
:1012E0001F9341E050E060E070E08A019B0104C080
:1012F000000F111F221F331F8A95D2F7C901B801B1
:101300001F910F910C945E090F931F9341E050E0E1
:1013100060E070E004C0440F551F661F771F8A9578
:10132000D2F78091730190917401A0917501B091F1
:1013300076018A019B01082B192B2A2B3B2BC90113
:10134000B8011F910F910C945E090F931F9341E018
:1013500050E060E070E004C0440F551F661F771F27
:101360008A95D2F74095509560957095809173015C
:1013700090917401A0917501B09176018A019B0151
:10138000082319232A233B23C901B8011F910F9178
:101390000C945E090F931F9341E050E060E070E011
:1013A00004C0440F551F661F771F8A95D2F780919E
:1013B000730190917401A0917501B09176018A0139
:1013C0009B01082719272A273B27C901B8011F912C
:1013D0000F910C945E090F931F930091730110916C
:1013E00074012091750130917601602B712B822B55
:1013F000932B1F910F910C945E090F931F930091F3
:101400007301109174012091750130917601602370
:101410007123822393231F910F910C945E090F93E4
:101420001F93009173011091740120917501309107
:10143000760160277127822793271F910F910C94C3
:101440005E0908952FE0929F800D1124E82FE69504
:10145000E695E695877051E001C0550F8A95EAF749
:1014600085E0E89FF0011124E85DFE4F20E030E0C8
:1014700070E04081CB01022E02C0969587950A94B8
:10148000E2F78170819584278523842781932F5FDC
:101490003F4F2530310569F708952FE0929F800D69
:1014A0001124682F669566956695982F977085E04C
:1014B000689FB001112440E050E080E0FB01E40FA0
:1014C000F51FE85DFE4F208130E0092E02C0369501
:1014D00027950A94E2F721703327042E01C0220FCA
:1014E0000A94EAF7822B4F5F5F4F4530510531F781
:1014F0000895BF92CF92DF92EF92FF920F931F93C6
:10150000CF93DF938C01C0907301D0907401E09071
:101510007501F09076018091770190917801A0910A
:101520007901B0917A01C82AD92AEA2AFB2ACFE1A7
:10153000D0E0D701C6010C2E04C0B695A7959795AB
:1015400087950A94D2F780FD04C0219790F7B12CBB
:1015500007C0BC2EB8018C2F0E94B4110197A9F3CB
:101560008B2DDF91CF911F910F91FF90EF90DF9026
:10157000CF90BF900895CF93DF93EC010E94790A3A
:10158000BE010E94B411DF91CF9108951F93CF93B4
:10159000DF93EB0190912701992321F0CB010E9469
:1015A000BB0A13C0882349F0CB010E94790A182F87
:1015B000682FCE010E94220A04C0CB010E944D0A6E
:1015C000182FBE01812F0E94B411DF91CF911F917E
:1015D00008951F93CF93DF93C0917B0116E0809114
:1015E0007C01C81799F0D0E01C9FF0011D9FF00D01
:1015F0001124E358FE4F40815181628173818481BF
:1016000095810E9402092196C770E9CFDF91CF91A1
:101610001F9108954091AD015091AE016091AF01CD
:101620007091B0018091B1019091B2010C940209C6
:10163000EF92FF920F931F93CF93DF938091B201AC
:1016400082958F7009F065C08091AF01882309F4FD
:1016500060C080917B01F0907C011091AD01009100
:10166000AE016091B0017091B10191E01F3F09F0AE
:1016700090E0C0916000D0916100292F96E0E92EA2
:101680008F1509F446C06115710521F00F3F21F057
:1016900030E003C031E001C0322F90E030FD36C0B1
:1016A000E89EF001E99EF00D1124DF01A358BE4F22
:1016B00011963C911197301329C03C91311326C0EB
:1016C00012963C911297311121C013964D915C9165
:1016D0001497461B570B4C175D07C0F48091B2015D
:1016E0008F7080618093B201EE57FE4F80818F70C2
:1016F000806180838DEA91E00E948408DF91CF9120
:101700001F910F91FF90EF900C94E90A019687705A
:10171000B7CFDF91CF911F910F91FF90EF90089578
:101720009F92AF92BF92CF92DF92EF92FF920F9370
:101730001F93CF93DF93CDB7DEB761970FB6F894C1
:10174000DEBF0FBECDBF8C0185E0F801DE011D9626
:1017500001900D928A95E1F7D8011296EC90909144
:10176000AD01E091AE012091B0013091B1012115A0
:10177000310531F0EF3F31F481E09F3F19F403C0B0
:1017800081E001C080E0B82FB1709B2E80FD47C181
:10179000D8014C9111965C9111971396AD90BC9025
:1017A00014978DEAC82E81E0D82EF090AF01B501D4
:1017B000621B730B2091600030916100FF2009F4DF
:1017C000D9C08091B2016217730708F095C0282F25
:1017D000207F09F052C05E1313C0491311C0FE2CC4
:1017E000E1100EC08F7080618093B2010E940A0BDD
:1017F000C6010E9484088091B201F80185834DC121
:10180000AB2831F05F3F31F481E04F3F19F403C062
:1018100081E001C080E080FD03C081E08E2502C030
:1018200080E090E0F82FF170FF2E80FF1CC08091C7
:101830007B0120917C0136E0821709F40BC190E016
:10184000389FF001399FF00D1124E358FE4F61815C
:10185000561306C06081461303C06281E61203C0BE
:1018600001968770E9CFFE2CEE2009F416C1809115
:10187000B20181608093B20154C05E1306C0491367
:1018800004C0E11002C0F80199C0C8010E94EB0831
:10189000882361F1EE2051F12091B201822F8295CF
:1018A0008F7090E0029774F08091AD019091AE013D
:1018B00098878F831986BB86AA862C87CE010796C8
:1018C0000E94840886E0F801ADEAB1E001900D9233
:1018D0008A95E1F70E94180B0E940A0B0AC05E1756
:1018E00011F1C8010E94EB0881112CC0C8010E94AF
:1018F0008408FF24F394D1C0282F207F81F77A2D0C
:10190000B98AA88A6E2D89890E94F3088DEA91E030
:101910000E94840886E0D6011D928A95E9F70E940C
:101920000A0BF12CBAC04913DCCFE110DACFF80171
:101930008583C8010E94840886E0D6011D928A959D
:10194000E9F7ABC0EE2091F22091B201822F82958F
:101950008F7090E002970CF4B5CF8091AD0190911B
:10196000AE019A8389831B82BD82AC822E83CE0115
:101970000196A6CF6217730708F044C0FE2CEE2034
:1019800009F4B4CF5E1330C049132EC02091B201C8
:1019900020FD21C0822F82958F70482F50E0411585
:1019A0005105C9F0F80125834F30510541F08F5F93
:1019B000982F9295907F822F8F70892B8583C801F5
:1019C0000E94840886E0F801ADEAB1E001900D9232
:1019D0008A95E1F73CC086E0F801ADEAB1E00190FC
:1019E0000D928A95E1F759C0C8010E94EB08811158
:1019F00069CF8091B20181608093B201C8010E94D9
:101A000084084BC07A2DB98AA88A6E2D89890E94D4
:101A1000F30886E0D6011D928A95E9F718C0EE20FA
:101A200009F464CFC8010E94EB08F82E882309F45A
:101A30005DCF86E0F801ADEAB1E001900D928A95A4
:101A4000E1F78DEA91E00E9493050E94180B0E9435
:101A50000A0B23C04D875E878D859E850E94BB0A39
:101A6000292F22952F70223028F49F7039F0811190
:101A700005C00BC0243028F49F7049F4805E883084
:101A800020F0C8010E9484089F2CF92C06C0D801C0
:101A900015969C91907F91F7F8CF8F2D61960FB698
:101AA000F894DEBF0FBECDBFDF91CF911F910F9194
:101AB000FF90EF90DF90CF90BF90AF909F900895F0
:101AC0001F93CF93DF93CDB7DEB72C970FB6F89463
:101AD000DEBF0FBECDBF4F83588769877A878B875C
:101AE0009C87CE0107960E94900B8823D1F09F819E
:101AF00088852A853B85232B31F08F3F31F481E0A7
:101B00009F3F19F403C081E001C080E080FD47C021
:101B10004F81588569857A858B859C850E9402094D
:101B20003EC086E0FE013796DE01119601900D92CF
:101B30008A95E1F7FF81E8856A857B8561157105E6
:101B400031F0EF3F31F481E0FF3F19F403C081E051
:101B500001C080E080FD23C020917C0130E0C901FC
:101B600001968770992740917B0150E08417950773
:101B7000F1F1F983EA837D836C8396E0929FD00133
:101B8000939FB00D1124A358BE4FFE0131960190D2
:101B90000D929A95E1F780937C010E94E90A16E084
:101BA00080917B0190917C01891771F1189FC00190
:101BB000112483589E4F0E94900B882329F1E091B5
:101BC0007B011E9FF0011124E358FE4F408151819B
:101BD00062817381848195810E94020980917B01D9
:101BE00090E001968770992780937B01D9CF0E945E
:101BF000CC0810927C0110927B01EDEAF1E086E0C6
:101C0000DF011D928A95E9F72C960FB6F894DEBF96
:101C10000FBECDBFDF91CF911F9108958091BB0181
:101C200085958595859508958091BB018770089568
:101C30009091BB01977081E009F480E00895809154
:101C4000C60108959091C601892B8093C60108951D
:101C500080959091C60189238093C60108951092C2
:101C6000C60108959091C501892B8093C5010895FF
:101C700080959091C50189238093C50108951092A4
:101C8000C50108958091BC01089508950C94450EF6
:101C90000C94460E9091940292FD08C09091BC0164
:101CA000981721F08093BC010C94480E0895809100
:101CB000BC01882329F01092BC0180E00C94480EEE
:101CC0000895CF93DF93E0916200F09163008091DB
:101CD000C6018083E0916200F09163009081809161
:101CE000C501892B80838091BC01882381F0E0911C
:101CF0006200F09163009081892B80838091620063
:101D0000909163000E945F2181110E94570EC09143
:101D10006200D091630048E050E063EB71E0CE01D7
:101D20000E94EE25892B69F088E0FE01A3EBB1E06B
:101D300001900D928A95E1F7CE01DF91CF910C943D
:101D40002821DF91CF9108950C94450E9091940233
:101D500092FD10C098E0899F90011124262B2093BA
:101D6000BB010E9484098091BB018595859585956D
:101D70000C94A40E0C9484091092BB0180E00C9486
:101D8000A40E2091BB01809582238093BB01982FE4
:101D9000977099F430E0482F082E000C550B24174B
:101DA000350759F09091940292FD07C0859585956D
:101DB00085950E94A5090C94BC0E089590919402FB
:101DC00092FB222720F9281769F080FB92F9909363
:101DD000940280919302909194020E94260F82E0D7
:101DE0000C94C10E08958091940282FB882780F99B
:101DF00091E089270C94DE0E81E00C94DE0E80E0E9
:101E00000C94DE0E80E090E00E94092621E0893EDD
:101E10009E4F09F020E0822F089582E090E00C941C
:101E2000FB2583E090E00C94FB25CF9384E090E0C9
:101E30000E94FB25C82F82E290E00E94FB252C2FF8
:101E400030E0A901582BCA01CF910895CF93C92F33
:101E5000682F84E090E00E940F266C2F82E290E0D1
:101E6000CF910C940F26AB01BC018FE090E00C9455
:101E70002026AB01BC0183E190E00C94202660E0B9
:101E800070E0CB010C94390F60E070E0CB010E9450
:101E9000330F0C943F0F69EE7EEF80E090E00E94DC
:101EA0002C2660E082E090E00E940F2660E083E054
:101EB00090E00E940F261092770110927801109204
:101EC000790110927A0160E084E090E00E940F2690
:101ED00060E082E290E00E940F2660E085E090E002
:101EE0000E940F2660E086E090E00E940F266FEFD0
:101EF00087E090E00E940F2640E050E0BA0188E0C1
:101F000090E00E94202660E08DE090E00E940F2685
:101F100040E050E0BA0188E190E00E94202660E0B5
:101F200087E190E00E940F2640E050E0BA018CE18A
:101F300090E00E94202660E070E080E290E00E9445
:101F40002C2640E050E0BA0188E190E00E94202673
:101F50000C94440F0C944B0F682F8EE090E00C947F
:101F60000F260E94EA216093DB017093DC018093CD
:101F7000DD019093DE016093D7017093D8018093C7
:101F8000D9019093DA01089584B7806884BF84B73B
:101F9000806884BF089581E008950C94CB0F089564
:101FA0000C94CF0F0C94CF0F0C94D20F0C94CF0F36
:101FB0000C94D60F0C94CF0F0E94C40F80E992E1CD
:101FC0000E9412210E94DA0F0C94D80F0E94D00FA9
:101FD0000C94CF0F0E9493120E9427050C94E91CC9
:101FE0000E94D7210E9478130E94EA0F0E94381B9A
:101FF0000E9477190C94D40F5F926F927F928F9208
:102000009F92AF92BF92CF92DF92EF92FF920F9387
:102010001F93CF93DF93CDB7DEB72A970FB6F8940F
:10202000DEBF0FBECDBF0E948D13C82E81110E944E
:10203000B10F37EC832E31E0932E00E010E0502EEC
:10204000802F0E94B7125C01F401619071904F01E2
:102050006826792661147104B1F40F5F1F4F0830B0
:10206000110569F78FEF89838A831B820E94DE2125
:102070008160782F9D838C8349815A816B818D810A
:102080000E9449053AC08091DF0181FD0E94C01283
:10209000D12CEE24E394F12CC3018E219F21892BB6
:1020A00029F10E94CD0F8823A9F0DE825F82AE2045
:1020B000BF2081E0AB2809F480E088870E94DE2100
:1020C0008160782F9A8789874E815F8168858A85AC
:1020D0000E944905000F111FF801E953FE4F80814E
:1020E0009181E826F926F182E08207C0D394EE0CB4
:1020F000FF1CFFE0DF12D0CFB0CF81E0C11001C0E4
:1021000080E02A960FB6F894DEBF0FBECDBFDF91F8
:10211000CF911F910F91FF90EF90DF90CF90BF90E4
:10212000AF909F908F907F906F905F9008950E94E6
:10213000FC0F0E94AA190E94E81C0C943E05CF9344
:10214000DF930E94B911EC01811522E59207E8F5B1
:10215000811531E5930708F0B6C0883E910528F552
:10216000803E910508F0E9C0883A910570F4853AFF
:10217000910508F07AC08130910509F473C008F424
:10218000D9C0049708F0D9C0D5C08F3B910508F09D
:10219000D1C0C85AD0E0CC0FDD1FCA54DF4F099020
:1021A000D881C02DCE019464C9C0811540E5940743
:1021B00008F069C0811550E4950708F060C09A9551
:1021C00081159F4108F4B9C0B5C0811536E5930764
:1021D00028F5811545E5940708F092C0811554E56E
:1021E000950708F087C0AC0143705527282F269526
:1021F0002695C115D34508F06CC081E090E002C07F
:10220000880F991F4A95E2F740E2249F900111241C
:10221000EC01C22BD32BCE019C6890C081152AE51E
:10222000920780F4811539E5930708F072C0811593
:1022300048E5940708F47EC0D82FCC27CE01806FE4
:10224000906A7CC090568115904208F073C08D2F23
:102250008F710E944D12DD27D0628F71AE01582B15
:10226000CA016CC081E090E069C0C55AD0E0CC5191
:10227000DF4F8881C82FD0E0CE0190645FC0DF704F
:10228000CE01906A5BC074E0969587957A95E1F7E8
:10229000282F23703C2F337081E090E002C0880F1C
:1022A000991F3A95E2F79C68AC01522B9A019C2F3A
:1022B0009F709695969550E2959FE0011124C90173
:1022C0008C2B9D2B3BC0D82FCC27CE01816F906AE1
:1022D00035C081E090E002C0880F991F4A95E2F76F
:1022E00050E2259F90011124EC01C22BD32BCE018B
:1022F0009A6824C0D82FCC27CE01846F906A1EC064
:102300000E944D128F7190E0D82FCC27CE019062A1
:1023100015C08F700E944D1294E0D695C7959A957E
:10232000E1F7CF70D0E0DC2FCC27D0699E01282BBD
:10233000C90104C080E090E001C0CE01DF91CF91DF
:10234000089528E7829FC0011124FC012FE0729FAD
:10235000E00DF11D1124E60FF11DEE0FFF1FE459F2
:10236000FF4F8591949108950E94A1110E949F10A2
:1023700008958238910569F1B0F48133910509F42B
:102380006DC048F48932910509F463C08A32910521
:1023900009F469C008958533910509F455C089335E
:1023A0009105B9F00895833E910569F138F4803EB6
:1023B0009105B1F0823E910509F10895863E91059F
:1023C000A9F1873E9105B9F1843E910509F064C0F9
:1023D00023C02091930220FD4FC021FD4DC00895E0
:1023E0008091930280FD44C08091940280FF44C09C
:1023F0008091930284FD42C083EE4DC08091930290
:1024000082FF38C0F5CF8091930282FD33C0809166
:10241000940280FD31C0ECCF8091940281FF32C0E4
:102420008091930284FD2AC087EE35C0809193028B
:1024300083FF26C0F5CF8091930283FD21C0809158
:10244000940281FD1FC0ECCF8091930285FD1CC0DA
:102450001DC08091930285FD19C016C08091930222
:1024600086FD16C017C08091930286FD13C010C070
:1024700089E311C082EE0FC080EE0DC080E00BC07A
:1024800086EE09C084EE07C089E205C085E303C07B
:102490008AE201C081E390E008959091930292FF57
:1024A0000DC0282F2871283019F4877F846006C05A
:1024B000282F2471243011F48B7F886093FF0DC086
:1024C000282F2871283119F4877E846106C0282FAF
:1024D0002471243111F48B7E88612091940220FFB5
:1024E0000DC0382F3871383019F4877F816006C0ED
:1024F000382F3171313011F48E7F886021FF0DC08B
:10250000282F2871283119F4877E816106C0282F71
:102510002171213111F48E7E886194FD877E0895AA
:1025200080E0089508950E94020F811102C00E9468
:10253000AA0F0E940D0F8093DF010E94150F909348
:102540009402809393020E9492120E94110F682FAE
:1025500070E080E090E00E94240960917301709126
:10256000740180917501909176010C945C09E82FBB
:10257000F0E0EE0FFF1FEB55FD4F80819181089534
:10258000089588E78A95F1F7089500C008950C949E
:10259000C11208950C94C9120C94CA120C94C91259
:1025A0000C94CE12F894E82FE295EF70F0E031A988
:1025B000282F2F7081E090E001C0880F2A95EAF75C
:1025C000982F9095932391AB92A9892B82AB789405
:1025D00008950F931F93CF93DF93C6EFD0E08991B7
:1025E0008F3F11F00E94D21280E0CE3FD807B9F79A
:1025F000C7EED0E006EF10E089918F3F11F00E9406
:10260000D2120C171D07C1F7DF91CF911F910F91C7
:102610000895BF92CF92DF92EF92FF920F931F9394
:10262000CF93DF938C01C62FD0E0CE018A509F4F0D
:102630006C01FC0190819F3F09F450C0B62EF894C4
:10264000E92FE295EF70F0E081A99F7021E030E082
:1026500001C0220F9A95EAF7822B81AB82A92095BF
:10266000282322AB78940E94C512E7EEF0E046EFF3
:1026700050E021E030E0E12CF12C61916F3F89F0D6
:10268000A62FA295AF70B0E0D0968C9190E06F70BD
:1026900002C0959587956A95E2F780FD02C0C90151
:1026A00002C080E090E0E82AF92A220F331F4E177B
:1026B0005F0719F7F60180818F3F11F00E94D21257
:1026C00061E0E114F10409F460E08B2D0E94C7126F
:1026D000CC0FDD1FC00FD11FF982E882DF91CF91AF
:1026E0001F910F91FF90EF90DF90CF90BF900895D2
:1026F0000E94E91280E1E5EAF2E0DF01982F1D92E5
:102700009A95E9F7E5E9F2E0DF011D928A95E9F78C
:1027100088E00E94D8130C948A04FF920F931F93B1
:10272000CF93DF93CDB7DEB760970FB6F894DEBFD7
:102730000FBECDBF8E010F5F1F4F80E1F8011192D8
:102740008A95E9F7F12C6F2DC8010E940913F394C3
:10275000F8E0FF12F8CF40E150E0B80185E992E0DF
:102760000E94EE25FF24F394009709F4F12C892BA5
:1027700041F080E1F801A5E9B2E001900D928A955F
:10278000E1F72F2D48E065EA72E085E992E00E94CA
:10279000D9130E948C048F2D60960FB6F894DEBF7B
:1027A0000FBECDBFDF91CF911F910F91FF90089584
:1027B0000895FF920F931F93CF93DF93F82E092F65
:1027C000162FD72FC42F222349F081E08093E201F6
:1027D0000E94DE219093E1018093E0018091E2016B
:1027E0008823D9F08091E0019091E1010E94F621C7
:1027F000059798F0EF2DF02FA12FBD2F80E090E0EE
:102800004C2F50E08417950734F4219131912D938A
:102810003D930196F7CF1092E201DF91CF911F9186
:102820000F91FF9008950E9440220E94F00F0C9497
:1028300051220E94CC210E9439220E94DC0F0E946A
:1028400013140E945F220E94E60FFBCFEF92FF92CB
:102850000F931F93CF93DF938B01682F11110AC041
:10286000442329F0E82FF0E0ED59FC4F6491762FD6
:10287000862F75C0212F30E0E82FF0E0442321F0AF
:10288000ED59FC4FE491F0E046E0049FC0011124B3
:10289000CFEFD0E0BE010E9454254BEA4603C001B1
:1028A000479F900D1124800F911D800F911D982F2F
:1028B000990F890FAE01421B530B4E9FD0014F9FC2
:1028C000B00D5E9FB00D11249B2F189FA001112405
:1028D000452F55278E01041B150B0E9FA0010F9F3E
:1028E000500D1E9F500D11247E01E81AF108E29E42
:1028F0008001E39E100DF29E100D1124212F33272D
:10290000C21BD30BCE9F9001CF9F300DDE9F300DA9
:10291000112462307105A9F048F46115710569F060
:1029200061307105C9F48B2F752F0DC064307105AE
:1029300081F058F06630710579F47E2F8B2F932F3C
:102940000DC0832F7B2F9E2F09C08E2F7B2F952F9D
:1029500005C08E2F732F02C07E2F852F692FDF9128
:10296000CF911F910F91FF90EF90089541E00E9449
:102970002614089508950E94B6140895CF93DF9306
:10298000762FE901682F842F0E94BB147983688316
:102990008A83DF91CF9108958091B502282F2695E3
:1029A00030E02115310519F48170826005C02532AF
:1029B000310524F0817088648093B502089588E021
:1029C00090E00C940326CF92DF92EF92FF926B017E
:1029D0007C010E94CC14B701A60188E090E0FF9032
:1029E000EF90DF90CF900C942026E5EBF2E083E0AF
:1029F000808311828FEF828383831482608171814F
:102A0000828193810C94E3148091B50280FF02C00F
:102A10008695089580E008959091B902933018F456
:102A20009F5F9093B902882351F06091B502709135
:102A3000B6028091B7029091B8020C94E314089505
:102A400081E00C940C159091B902992319F09150E2
:102A50009093B902882351F06091B5027091B6024B
:102A60008091B7029091B8020C94E314089581E02C
:102A70000C94231570E00C94F51C60916800809113
:102A8000B50280FF0AC08091670023E0829FC001E9
:102A9000112486549D4F0C943A15809169009091B1
:102AA0006A00891780F7E82FF0E09F01220F331F9B
:102AB000E20FF31FE654FD4F1182108212828F5FE6
:102AC000F0CF9091B50290FF16C0909169002091CF
:102AD0006A00921770F4E92FF0E0DF01AA0FBB1F24
:102AE000EA0FFB1FE654FD4F8183608342839F5FA3
:102AF000F0CF0C943D150895CF93DF9300D01F9233
:102B0000CDB7DEB79091B50290FF0AC09E012F5F4E
:102B10003F4F0E94BE144B8169818A810E946115DA
:102B20000F900F900F90DF91CF910895CF93DF9387
:102B3000EC01EC81F0E0E25AFD4F4491E5EBF2E06C
:102B4000628181810E947C158C818F5F8C83DF91F3
:102B5000CF910895CF93DF93EC01E5EBF2E0438151
:102B600062818C810E947C158C818F5F8C83DF91C8
:102B7000CF9108950F931F93CF93DF9300D01F92AF
:102B8000CDB7DEB78C018091E30181110AC09E01AF
:102B90002F5F3F4F4FEF6FEF0E94BE148A818093EB
:102BA000E301F8018481813051F028F0823061F432
:102BB0004091E3010AC08091E30140E007C06091C9
:102BC000E30140E080E003C040E080E060E00E947C
:102BD0006115F801848190E0019663E070E00E9445
:102BE000682584830F900F900F90DF91CF911F91F4
:102BF0000F910895AF92BF92CF92DF92EF92FF9222
:102C00000F931F93CF93DF9300D01F92CDB7DEB702
:102C1000182FF62E042FE22E9091B50290FF6DC072
:102C2000E92FE695AE2FB0E0A250BF4F8C91809374
:102C3000ED019E7F923061F49E012F5F3F4F812F07
:102C40000E94BE144B8169818A810E94611543C034
:102C5000823019F40091B8023EC0863019F4109108
:102C6000B60239C08930D9F38931A9F5E9518E2FDF
:102C70008170D82EE695F0E0E25AFC4FA590B49012
:102C8000C12CBB2460916B00C61618F52C2D30E0CA
:102C9000A29EC001A39E900DB29E900D112470E0E3
:102CA0000E945425812FD11002C0860F01C0861BBF
:102CB00090916900290F311DA901440F551F240F60
:102CC000351F26543D4F402F6F2D0E94BE14C394D4
:102CD000D9CF0E943D151093B602F092B70200932F
:102CE000B802EE2051F06091B5027091B602809169
:102CF000B7029091B8020E94E3140F900F900F90CA
:102D0000DF91CF911F910F91FF90EF90DF90CF90C7
:102D1000BF90AF900895E5EBF2E09181282F4381B9
:102D2000628188E0890F0C94FA1581E00C948B166F
:102D3000E5EBF2E09181282F4381628188EF890FD2
:102D40000C94FA1581E00C949816E5EBF2E06281A0
:102D500021E1620F08F46FEF282F438181810C94E9
:102D6000FA1581E00C94A516E5EBF2E0628121E111
:102D7000621B08F460E0282F438181810C94FA15CE
:102D800081E00C94B416E5EBF2E0438121E1420FBF
:102D900008F44FEF282F628181810C94FA1581E0AD
:102DA0000C94C316E5EBF2E0438121E1421B08F4E9
:102DB00040E0282F628181810C94FA1581E00C9407
:102DC000D21620E00C94FA15FF920F931F93CF9325
:102DD000DF93EC01F12C0FEF10E060916B00F61621
:102DE000F0F4809169002F2D30E0280F311DC901CA
:102DF000880F991F280F391F26543D4F70E0C801D6
:102E00000E946825962F8C814091B8026091B7028C
:102E1000F99E800D11240E94BE14F394DECF0E940F
:102E20003D159A818C8190FF02C08F5F01C0815057
:102E30008C83DF91CF911F910F91FF900895AF92F6
:102E4000BF92CF92DF92EF92FF920F931F93CF9397
:102E5000DF93FC01828180FF02C00FEF01C001E01F
:102E600010E045E0A42E80916B00181708F043C0D5
:102E700080916900C12ED12CE601C80FD11DCE0171
:102E8000880F991FC80FD91FC654DD4F19821882A9
:102E90001A8234E0E32EF12CB12C8091E5018B0DE8
:102EA00086302CF06A2D0E944625892F05C087FFA9
:102EB00003C090916B00890F082E000C990BC81667
:102EC000D90691F48091B8028E9DA0018F9D500D7E
:102ED000112455954795559547959E016091B702E8
:102EE0008091B6020E94BE14B00EF1E0EF1AF10814
:102EF000A1F61F5FB8CF0E943D158091E50101301A
:102F000031F4811102C080916B00815007C090E0C4
:102F1000019660916B0070E00E9468258093E50146
:102F2000DF91CF911F910F91FF90EF90DF90CF90A5
:102F3000BF90AF900895CF938091690090916A00FF
:102F4000891770F4E82FF0E09F01220F331FE20F82
:102F5000F31FE654FD4F1182108212828F5FF0CF73
:102F6000C0E060916B00C617C0F5EC2FF0E070E098
:102F7000CF010E94682520916900820F2091E40111
:102F8000022E000C330B90E0E217F307CCF02091F7
:102F90006600022E000C330B2E173F078CF09C01AD
:102FA000220F331F820F931F9C0126543D4F4091E7
:102FB000B8026091B7028091B6020E94BE140BC0A5
:102FC000FC01EE0FFF1F8E0F9F1FFC01E654FD4F0B
:102FD000118210821282CF5FC4CF0E943D152091D2
:102FE00065008091E401820F8093E4019091660076
:102FF000920F9093660019165CF4082E000C990B42
:1030000040916B0050E041505109841795071CF026
:10301000219520936500CF9108958F929F92AF9252
:10302000BF92CF92DF92EF92FF920F931F93CF93B5
:10303000DF938C01FC014481C42FD0E09E01DE01AE
:103040000E94AC259B01AC010E94C2256B017C0152
:10305000E0E2F0E0EC1BFD0BA5E5B0E09B01AC016C
:103060000E94C2254B015C019F01DF010E94A42543
:103070009B01AC010E94CD259B01AC012C0D3D1D97
:103080004E1D5F1DC501B4010E947C25C22FD22FA9
:103090002A3228F4F3E02F9F900111240DC025E57A
:1030A00030E02C1B3109C901880F991F280F391FE7
:1030B00037FF02C02F5F3F4F35952795C22FC09530
:1030C000F12C85E5E82EED1A80916B00F816C8F416
:1030D000F1FC02C08E2D01C08D2F909169002F2D23
:1030E00030E0290F311DA901440F551F240F351F52
:1030F00026543D4F4C2F6091B7020E94BE14F394AA
:10310000E3CF0E943D15F8018481811102C091E056
:1031100003C0803219F49FEF909364009091640093
:10312000890FF8018483DF91CF911F910F91FF9058
:10313000EF90DF90CF90BF90AF909F908F900895C9
:103140000F931F93CF93DF93EC0100E010E0809189
:103150006B00282F30E00217130724F590916900C7
:103160009801290F311DA901440F551F240F351F48
:1031700026543D4F869590E04C81081719071CF4A2
:10318000442331F002C0411103C04091B80201C094
:1031900040E06091B7028091B6020E94BE140F5FBA
:1031A0001F4FD5CF0E943D158C8190E00196817014
:1031B00099278C83DF91CF911F910F910895E5EBB3
:1031C000F2E080818E7F8083608171818281938132
:1031D0000E94E3141092EE012FEB84ED91E0215058
:1031E00080409040E1F700C000000C943D156091D4
:1031F000B502669570E04BE050E08CE690E00E94EE
:10320000E125892B19F481E08093EE010E94DE21F3
:103210009093E7018093E60108959091B50290FFA5
:1032200035C09170811102C0926006C0853210F0E5
:10323000986402C0880F982B9093B502662351F0D2
:103240006091B5027091B6028091B7029091B80278
:103250000E94E3146091B502669570E04BE050E087
:103260008CE690E00E94E125892B19F01092EE0186
:1032700002C00E94F71881E08093E9014091B802F2
:103280006091B7028091B6020C94E1160895682F00
:103290009091B502969581E0890F853208F081E022
:1032A0000C940D1981E00C944719682F9091B50288
:1032B00096958FEF890F09F484E20C940D1981E043
:1032C0000C94551961E00C940D19E5EBF2E0808146
:1032D0008160808386950C9462198091B50280FD8F
:1032E0000C94DF180C94651960E00C940D19809112
:1032F000EC0181112EC00E94020F811104C00E94B6
:10330000AA0F0E94F5140E94DF146093B502709317
:10331000B6028093B7029093B8026E7F61F40E9468
:10332000F5140E94DF146093B5027093B602809387
:10333000B7029093B8020E94CC141092EE018091D3
:10334000B50280FF03C086950E94741981E08093C6
:10335000EC0108950F931F93CF93DF938091EE01BB
:10336000882309F485C08091ED01E091B502E695CE
:10337000E81BE093E801823049F4F0E0E65AFD4FA3
:10338000E491CE2FD0E006E915E149C0863049F43A
:10339000F0E0E95AFD4FE491CE2FD0E00AEA15E1C2
:1033A0003EC0893051F4E695F0E0EC5AFD4FE491CF
:1033B000CE2FD0E004EE16E132C08F3051F4E69506
:1033C000F0E0EF5AFD4FE491CE2FD0E00FE117E18E
:1033D00026C0853149F4F0E0E25BFD4FE491CE2F49
:1033E000D0E00BE917E11BC0883181F0833239F45A
:1033F000ECE4F2E0C591D4910AEB15E110C08432FF
:1034000051F4C4EFD1E000EA18E109C0C8E2D0E00D
:103410000DE018E104C0C0EDD7E00AEB14E18091A3
:10342000E901882361F01092E9010E94DE21909366
:10343000E7018093E6011092EB011092EA010E94ED
:10344000DE21E091E601F091E7018E1B9F0B8F3F9B
:103450009F4770F4EC0FFD1FF093E701E093E60146
:1034600086EE91E0F801DF91CF911F910F910994C1
:10347000DF91CF911F910F910895882311F0FA01E8
:1034800001C0FB010994CF93DF93C82FD62F0E9470
:1034900004158C1740F00E9404158D1720F4DF915D
:1034A000CF910C9452198C2FDF91CF910C9462190B
:1034B0001F93CF93DF93FB0112811111C3C0EC0165
:1034C0000E941F0E8272CD3CFCE5DF0709F49AC012
:1034D000A8F5C73CECE5DE0709F476C0A8F4C43CC7
:1034E0009CE5D90709F45FC028F4C33CDC4509F426
:1034F00057C054C0C53C9CE5D90709F459C0C63C27
:10350000DC4509F45CC04AC0CA3CFCE5DF0709F4AD
:103510006AC050F4C83CECE5DE0709F45AC0C93C67
:10352000DC4509F45BC03AC0CB3C9CE5D90709F403
:103530005FC0CC3CDC4509F460C030C0C23DFCE556
:10354000DF0709F46FC088F4CF3C9CE5D90709F484
:1035500060C008F45CC0C03DFCE5DF0709F45CC056
:10356000C13DDC4509F45BC019C0C53D9CE5D907E8
:1035700009F460C050F4C33DFCE5DF0709F455C011
:10358000C43DDC4509F454C009C0C63D9CE5D907DB
:1035900009F455C0CE35DD4509F454C011E052C0E0
:1035A0000E946D194FC04FE559E162E579E104C011
:1035B00042E559E16FE579E10E943D1A43C042EAD4
:1035C00056E165E976E1F8CF45E956E162EA76E150
:1035D000F3CF40EC56E161EB76E1EECF41EB56E103
:1035E00060EC76E1E9CF4EED56E16FEC76E1E4CFA9
:1035F0004FEC56E16EED76E1DFCF47E355E160E257
:1036000075E1DACF40E255E167E375E1D5CF81E0BE
:1036100017C065E082E010C068E086E00DC06EE093
:1036200089E00AC064E18FE007C067E185E104C07A
:1036300088E106C062E289E10E94431A03C083E286
:103640000E946219812FDF91CF911F91089586E02A
:1036500090E00C94FB25682F86E090E00C940F26F8
:103660008091C902847089618093C9020C942B1BDC
:103670000E94020F811104C00E94AA0F0E94301BF9
:103680000E94271B8093C902282F269526952695F0
:1036900030E02430310524F0877088618093C902BE
:1036A0008091C90280FF04C086958695869501C0E9
:1036B00080E00C94491C2091C902822F8695869542
:1036C0008695482F50E04330510554F48F5F982F72
:1036D000990F990F990F822F8770892B8093C902B8
:1036E0008091C90281608093C9020E942B1B809146
:1036F000C9028695869586950C94491C8091C902CD
:10370000982F969596959695A1F0915E990F990FA1
:10371000990F8770892B8093C902887F91E009F403
:1037200090E08091C90290FB80F98093C9020E94C9
:103730002B1B8091C9028695869586950C94491C11
:103740008091C90280FD13C081608093C9028130DD
:1037500019F489E08093C9028091C9020E942B1B51
:103760008091C9028695869586950C94491C08958A
:103770008091C90280FF08C08E7F8093C9020E9499
:103780002B1B80E00C94491C08958091C90280FD98
:103790000C94B81B0C94A01B9091C902892F86959C
:1037A000869586958F5F8F719770843038F4880F77
:1037B000880F880F892B8093C90202C09093C90299
:1037C0008091C902887F91E009F490E08091C9025C
:1037D00090FB80F98093C9020E942B1B8091C90243
:1037E0008695869586950C94491C843008F083E074
:1037F0009091C9029770282F220F220F220F922B2F
:103800009093C902987F21E009F420E09091C902C9
:1038100020FB90F99093C9020C94491C0E94F51B5F
:103820008091C9020C942B1B9C01FB01828188238F
:1038300049F12E3BFCE53F07C9F040F42C3BECE599
:103840003E0769F02D3B3C4561F00895203C9CE526
:10385000390791F070F0213C3C4589F0089583E0F0
:1038600001C080E00E940E1C80E008950E947E1B33
:10387000FBCF0E945B1BF8CF0E94C51BF5CF0E94B7
:10388000CC1BF2CF81E008958C9A94980895949877
:1038900008958F929F92AF92BF92CF92DF92EF9254
:1038A000FF920F931F93CF93DF93C82F843040F480
:1038B000811107C08FB58F7D8FBD0E94471C04C04A
:1038C000C3E08FB580628FBDA6B5B7B52C2F30E0B1
:1038D0000E94AC2523E030E040E050E00E947C25CF
:1038E0000027122F232F342F012F122F232F33279E
:1038F00086B597B56CE070E00E945425601771079B
:1039000030F0C80169E070E00E94542552C086B5CD
:1039100097B5E6B4F7B4E6B5F7B5C6E0D0E0BE01BA
:103920000E945425060F171F211D311D4801590102
:1039300085E0880C991CAA1CBB1C8A95D1F7C7018D
:10394000BE010E9454256F01E12CF12CA7019601C4
:10395000260F371F411D511DC501B4010E947C2552
:1039600069017A01E6B5F7B5CA01B9010E943625A9
:103970009B01AC01DF010E94C2259B01AC01C70184
:10398000B6010E943625DC01CB012FE0B695A79544
:10399000979587952A95D1F706B517B520E030E0C1
:1039A000081719072A073B0718F466B577B5CB0146
:1039B000BC0179BD68BDDF91CF911F910F91FF9040
:1039C000EF90DF90CF90BF90AF909F908F90089531
:1039D00008950E94441C82E28FBD89E18EBD8FEF65
:1039E0009FEF97BD86BD0C94381B0F931F93CF9309
:1039F000DF938C01EB018091EF01811105C00E94E2
:103A0000392081E08093EF01AE01440F551F4C0F28
:103A10005D1F24E630E0B80180EBDF91CF911F916C
:103A20000F910C94EC20CF93DF93EC01FB0182818A
:103A3000882309F43CC1C430FDE5DF0760F4CB3FC7
:103A40009CE5D90788F49E0122503C45243131057C
:103A500008F02EC109C0C236EDE5DE0729F0C63AEE
:103A6000FDE5DF0709F024C10E94150F9093940231
:103A700080939302C1318CE5D80709F4C6C008F0E1
:103A800042C0C930ECE5DE0709F49BC000F5C53043
:103A90008CE5D80709F485C078F4C330ECE5DE077F
:103AA00009F478C008F07AC0C230DC4509F0F5C0EE
:103AB000809193028160EFC0C7309CE5D90709F47B
:103AC00078C008F07AC0809193028061E4C0CD3064
:103AD000FCE5DF0709F487C058F4CB309CE5D90733
:103AE00009F479C008F07BC08091930288606FC0B0
:103AF000CF30FCE5DF0709F480C008F082C0809178
:103B00009302877FC8C0CE3F9CE5D90709F471C0F6
:103B100000F5C531FCE5DF0709F485C068F4C33161
:103B20009CE5D90709F475C008F095C00E94CC083F
:103B3000809193028F77AFC0CC3FFCE5DF07A9F1FE
:103B400008F054C0CB3FDC4509F0A7C08091940237
:103B500040C0C230EDE5DE0709F489C058F4C11554
:103B60008DE5D80709F45AC008F069C08091940225
:103B700082602FC0C236EDE5DE0709F47CC0C63A8C
:103B8000FDE5DF0709F481C0C330DD4509F085C0DC
:103B900080E06EC08091930282607DC0809193022C
:103BA00016C080919302886076C0809194028260F2
:103BB0004FC08091930280626EC0809193028064B6
:103BC0006AC00E94CC0880919302806864C08460BF
:103BD00062C081603DC0809193028E7F5CC0809105
:103BE00093028D7F58C08091930216C080919402F9
:103BF00018C0809194028D7F2BC0809193028F7E9C
:103C00004AC0809193028F7D46C0809193028F7B42
:103C100042C080919302877F8B7F3DC08091940248
:103C20008D7F8E7F15C08091930282FB222720F921
:103C300091E0922790FB82F990FB83F92CC0809150
:103C40009402982F909591708E7F892B90FB81F92B
:103C50008093940222C00E94CC088091930287FB3B
:103C6000222720F991E0922790FB87F914C081E088
:103C70000E94AC0F12C08091930284FB222720F98E
:103C800091E0922790FB84F906C080919302982FCF
:103C9000909590FB80F9809393028091930290918C
:103CA00094020E94260F0E94CC0880E001C081E0AF
:103CB000DF91CF9108950F931F9341E050E060E0B2
:103CC00070E08A019B0104C0000F111F221F331FE7
:103CD0008A95D2F7C901B8010E9424091F910F915A
:103CE0000C94CC088B3109F468C058F58B3009F47A
:103CF00086C078F4863009F445C020F4853009F494
:103D00004BC07FC0873009F44AC0883009F477C0BF
:103D100078C0803109F464C068F48E3009F071C055
:103D20008091DF0182FB222720F991E0922790FB0E
:103D300082F94CC0863109F462C0893109F45FC050
:103D400060C08A32E1F060F4873209F455C028F48B
:103D50008E3108F456C08D5150C08932E9F051C0FF
:103D6000833450F48A3308F045C0853309F444C0E5
:103D7000883309F444C045C08334F1F142C00E9445
:103D8000AA0F3DC08091DF01817F8E7F8093DF018C
:103D900081E08093F00108950E948F0430C08091EB
:103DA000DF01982F9095917090FB80F98093DF014F
:103DB000911125C0897F877F10C08091DF0181FB31
:103DC000222720F991E0922790FB81F98093DF016F
:103DD0009923A9F08091DF0181608093DF010FC0FA
:103DE0008091DF0183FB222720F991E0922790FB4D
:103DF00083F9ECCF895301C080E00E945B1E81E013
:103E0000089580E0089580E008950C94031FCF93F7
:103E1000C82F8091F001882319F0813031F02BC038
:103E20000E941F0E823249F504C00E941F0E82328A
:103E300061F48C2F0E94051F811104C08C2F0E94F9
:103E4000721E17C081E090E014C08C2F0E94031FE7
:103E500081110EC0C43149F018F4CB3049F00FC0C5
:103E6000C93219F0C83321F00AC01092F00107C01E
:103E700081E0817006C01092F00180E002C080E015
:103E8000F8CFCF910895CF93DF9386319C4541F5CC
:103E9000EB010E941F0E982F8A81209162003091C1
:103EA0006300882379F09A7A81E009F480E08093B6
:103EB000F101911102C069E201C065E3C9010E94EC
:103EC000A1210AC08091F101811102C069E201C003
:103ED00065E3C9010E94A3210E94610E80E001C038
:103EE00081E0DF91CF9108950F931F93CF93DF93DC
:103EF000C42FD22FFC0182818823C9F04093F401A2
:103F00000E94DE219093F3018093F20180E28C0FF6
:103F1000883008F057C0C77081E001C0880FCA958B
:103F2000EAF7DF91CF911F910F910C9438068091A1
:103F3000F401481330C08091F2019091F3010E9486
:103F4000F621883C910538F510E21D0FCD17B9F028
:103F500080E28C0F883040F4C77081E001C0880F88
:103F6000CA95EAF70E943F06183028F581E09D2F98
:103F7000977001C0880F9A95EAF70E943806802F43
:103F80000E942F061830F0F4D77081E001C0880F2E
:103F9000DA95EAF70AC080E28C0F883098F4C7708F
:103FA00081E001C0880FCA95EAF7DF91CF911F9198
:103FB0000F910C943F06802FDF91CF911F910F91AD
:103FC0000C942F06DF91CF911F910F9108950F93BD
:103FD0009C01CB01243F4CE5340731F188F4293DA5
:103FE000FCE53F07D9F02A3D4CE5340779F1283D3F
:103FF0003C45A9F506E221EE41EE68ED7CE52BC0DB
:10400000263FFCE53F07E1F0A8F0273F3C4539F5A6
:1040100007E225EE46EE67EF7CE51DC007E225EEE0
:1040200045EE69ED7CE517C006E221EE40EE64EF57
:104030007CE511C007E225EE44EE65EF7CE50BC0A0
:1040400006E221EE42EE66EF7CE505C008E221E0E3
:1040500045EE6AED7CE50E94741F80E008C0FC011B
:104060008281882319F01092F40101C081E00F9140
:10407000089511B887E080B985B3836085BB86B7A2
:10408000846086BF86B7816086BF86B7806486BF3E
:1040900008959F92AF92BF92CF92DF92EF92FF92DC
:1040A0000F931F93CF93DF93B82EEB010E94DE2175
:1040B0006C01C431D10558F0CF3F8FEFD80759F0CC
:1040C000CE0164E170E00E9454257B0107C0EE241C
:1040D000E394F12C03C025E0E22EF12C84E8A82E15
:1040E00094EA992E16BE96BE0E94DE218C0106B679
:1040F00007FC08C00E94DE21801B910B8E159F05D6
:10410000B0F324C081B1887F883039F081B1887FD5
:10411000803119F00FEF1FEF1BC0B3B8A6BE0E948D
:10412000DE218C0106B607FC08C00E94DE21801B40
:10413000910B8E159F05B0F309C081B1887F88313E
:1041400011F0803439F700E010E00DC00EEF1FEFE2
:10415000CF3F8FEFD80731F2C6010E94F6218C17AE
:104160009D0708F4BFCFC801DF91CF911F910F9138
:10417000FF90EF90DF90CF90BF90AF909F90089509
:104180000F931F93CF93DF93EB0183B984E886BF2E
:104190000E94DE218C0106B607FC0EC0CF3F8FEFD8
:1041A000D807C9F30E94DE21801B910B8C179D0755
:1041B00090F38EEF9FEF0BC021B1287F81E090E05C
:1041C000283211F480E090E0919581959109DF917A
:1041D000CF911F910F910895CF92DF92EF92FF92AE
:1041E0000F931F93CF93DF936B018A017901B9017C
:1041F0000E944920E6010C0D1D1DC017D10759F47E
:1042000024E926BFDF91CF911F910F91FF90EF908E
:10421000DF90CF90089597FDF3CFB70189910E9469
:10422000C020EBCF909325018093240108959093B3
:10423000FA018093F9010895E091F901F091FA01F2
:10424000309721F00190F081E02D099480E00895ED
:10425000E091F901F091FA01309721F00280F381A9
:10426000E02D099408952091F7013091F801281765
:10427000390771F09093F8018093F701E091F9010B
:10428000F091FA01309721F00680F781E02D099432
:1042900008952091F5013091F6012817390771F042
:1042A0009093F6018093F501E091F901F091FA0104
:1042B000309721F00084F185E02D09940895FC01E8
:1042C000329697E080E0915029F021912223D9F392
:1042D0008F5FF9CF0895662349F0FC013296089666
:1042E0002191621729F0E817F907D1F780E00895C6
:1042F00081E008959C01FC0132969FEF80E041919E
:10430000461789F09F3F19F4411101C0982F8F5F24
:104310008630A9F79F3F39F0F901E90FF11D97FDAC
:10432000FA956283089508959C012A5F3F4FFC012E
:104330004281461301C01282019682179307B9F792
:1043400008950C947A210C949421029626E0FC01A5
:1043500011922A95E9F7089508950C94AC210C94D4
:10436000AD210C94AC210C94AC210C94AC21CF93D6
:104370000E94B3210E948D130E94B121C0E08C2FB6
:104380000E94B712892B29F4CF5FC830C1F780E0B3
:1043900001C081E0CF91089508958091FD018111C0
:1043A0000C94FE0408950E94CC080C9405058BE043
:1043B00083BF8BEB8CBF82E089BF08952FB7F89441
:1043C0008091CA029091CB02A091CC02B091CD0213
:1043D0002FBF08952FB7F8946091CA027091CB0255
:1043E0008091CC029091CD022FBF08959C014FB7D0
:1043F000F8948091CA029091CB02A091CC02B09126
:10440000CD024FBF821B930B089578941F920F9299
:104410000FB60F9211248F939F93AF93BF93809108
:10442000CA029091CB02A091CC02B091CD0201962C
:10443000A11DB11D8093CA029093CB02A093CC0220
:10444000B093CD02BF91AF919F918F910F900FBE0E
:104450000F901F90189560E081E090E00E94322656
:104460009CE088E10FB6F894A89581BD0FBE91BD80
:10447000FFCF0E94DE219093FC018093FB01089501
:104480000E941B258B9A80E0815041F0A895E7EBB4
:10449000FBE03197F1F700C00000F6CF8B987894DD
:1044A00008950E943E230E9417212FEB84ED91E096
:1044B000215080409040E1F700C0000008958091B5
:1044C000F502882389F01092F5020E94DE21909374
:1044D000FC018093FB018091FD018823D1F11092B2
:1044E000FD010E94D32111C08091FD01811111C0F5
:1044F0008091FB019091FC010E94F621069728F023
:1045000081E08093FD010E94CD218091FD018823EF
:1045100001F10E94CD210E94B721882339F1F8943E
:1045200021B3939A822F8C6081BB92B38CE0982741
:1045300092BB3FE54AEE90E0315040409040E1F7B9
:1045400000C0000092B3892782BB21BB9398789466
:1045500008950E9424248091FB02882329F08091F1
:10456000D90284FD0E9497100C94E5220895809151
:1045700092020895089590910302981307C0209124
:1045800001023091020226173707A9F08093030237
:1045900070930202609301028093FE017093000207
:1045A0006093FF018091120384FF05C063E08EEFEA
:1045B00091E00C9420240895BC0184E00C94BB226B
:1045C000BC0183E00C94BB220895CF93DF93CAE033
:1045D000D0E08091D90284FF18C080910F029091A1
:1045E00010029817E1F028E0829FC001112468E0D2
:1045F0008F5E9D4F0E941C2480910F0290E00196D7
:104600008F70992780930F020AC00E94242487EBA1
:104610009BE00197F1F700C000002197D1F6DF91F0
:10462000CF910895CF93DF93EC01A0911002B0E0F9
:10463000CD0101968F70992720910F02281779F0EC
:1046400093E0AA0FBB1F9A95E1F7AF5EBD4F98E0CC
:10465000FE0101900D929A95E1F7809310020E945D
:1046600024240E94E52288E0FE01A7E0B2E0019048
:104670000D928A95E1F7DF91CF91089587E790E059
:104680000895FC01808180768032A1F5818181309E
:1046900061F484819581892B69F587E092E090939C
:1046A000F7028093F60288E00895823041F481E9B0
:1046B00092E09093F7028093F60281E008958A30A9
:1046C00021F483818093910215C0893099F482810D
:1046D00093818115924081F484819581892B61F4C5
:1046E00081E08093060286819781909305028093F2
:1046F000040202C080E008958FEF08952091040223
:1047000030910502232B71F020910602213051F4E3
:10471000FC018081809392021092050210920402A3
:1047200081E008958FEF08950895FC0193819330FF
:10473000D9F068F4913081F0923009F059C083E6E5
:1047400094E09093F7028093F6028BE30895913200
:1047500049F19232B9F14CC08EE994E09093F7029E
:104760008093F60282E108958281813099F050F0C1
:104770008230F1F580EB94E09093F7028093F6029B
:104780008AE0089586ED94E09093F7028093F60214
:1047900084E008958CEB94E09093F7028093F60206
:1047A00088E108958281882329F0813009F58EE817
:1047B00094E002C085E794E09093F7028093F602BC
:1047C00089E0089584819581009751F0019781F4E3
:1047D0008AED94E09093F7028093F60282E30895C5
:1047E0008CE095E09093F7028093F60280E40895C0
:1047F00080E008951F93CF93DF93162FEA0128815D
:1048000024FF05C0398128E82327298302C02AE52F
:104810002883212FFC01CE010296DC0131913D93CA
:1048200021501216DCF3612F0E94DA021C5F1883FC
:10483000DF91CF911F91089549ED52E00C94FA2336
:1048400042E153E00C94FA23CF93DF936091F80296
:10485000635067FD93C08091F402CCE0D0E0C81BA8
:10486000D109C450DD4F8091F302803120F4CE0194
:104870000E94942381C08D3209F06EC0683009F027
:104880007BC083EC8093CE028AE5809384001092F3
:10489000F2028881807621F0CE010E94412349C036
:1048A0009A811092D7028981811106C01092D80294
:1048B00027ED32E082E038C0853019F49093F90298
:1048C00030C08630A1F48B81813041F0823031F0EC
:1048D000833021F0813211F0823221F4CE010E9426
:1048E000952301C080E090E49093F20222C08830CA
:1048F00089F0893019F49093FB0213C08A3069F073
:104900008B3079F48BE48093DA02809313038093E5
:10491000E60207C02BEF32E002C027ED32E081E073
:1049200003C027ED32E080E03093F7022093F602D7
:1049300009C08F3F39F4988197FD8E8190E890935C
:10494000F20207C09F81911104C09E81981708F45C
:10495000892F8093830010C08091F20287FF0CC0E2
:10496000CE010E947E238F3F21F48EE1809384004C
:1049700003C08111109283001092F802809184008C
:1049800084FF4CC0809183008F3F09F447C0C82F3B
:10499000893008F0C8E08C1B809383009091CE0290
:1049A00088E889278093CE02CC2359F18091F602C2
:1049B0009091F7022091F20226FF12C0AEECB2E015
:1049C0002C2FAC014E5C5240FA01EA0FFB1FE49120
:1049D0001196EC931197215011962111F5CF08C033
:1049E000EFECF2E0DC012C2F3D9131932150E1F707
:1049F00001962FEF2C0F820F911D9093F702809359
:104A0000F6026C2F8FEC92E00E94DA02CC5FCC3081
:104A100019F08FEF80938300C093840084E190B3FA
:104A20009C7031F48150D9F71092F9021092F10282
:104A3000DF91CF910895CF93DF9385B7886085BFCD
:104A40008BB780688BBFC9EDD2E08BE48983A2E18C
:104A5000B3E011968C931197E5EEF2E081838AE53D
:104A600088838C938083DF91CF910895DB018F93AE
:104A70009F930E94C225BF91AF91A29F800D911D6F
:104A8000A39F900DB29F900D1124089587FB082ECF
:104A9000062687FD819567FD61950E94D5250EF458
:104AA000919507FC81950895AA1BBB1B51E107C096
:104AB000AA1FBB1FA617B70710F0A61BB70B881FAE
:104AC000991F5A95A9F780959095BC01CD0108953D
:104AD00097FB072E16F4009407D077FD09D00E94AB
:104AE000542507FC05D03EF4909581959F4F08957D
:104AF000709561957F4F0895A1E21A2EAA1BBB1BEA
:104B0000FD010DC0AA1FBB1FEE1FFF1FA217B30799
:104B1000E407F50720F0A21BB30BE40BF50B661FAF
:104B2000771F881F991F1A9469F760957095809573
:104B300090959B01AC01BD01CF010895EE0FFF1FC1
:104B40000590F491E02D09940E94AC25332312F4D2
:104B50008A1B9B0B0C94BD25A29FB001B39FC00183
:104B6000A39F700D811D1124911DB29F700D811D99
:104B70001124911D08950E94AC25B7FF0895821B52
:104B8000930B08950E94AC25A59F900DB49F900DA6
:104B9000A49F800D911D11240895B7FF0C94C22588
:104BA0000E94C225821B930B0895991B79E004C0D3
:104BB000991F961708F0961B881F7A95C9F780955C
:104BC0000895FC014150504030F001900616D1F795
:104BD0003197CF010895882799270895FB01DC01BB
:104BE00004C08D910190801921F441505040C8F7C4
:104BF000881B990B0895E199FECF9FBB8EBBE09A6D
:104C000099278DB30895A6E1B0E044E050E00C94FC
:104C10004126A8E1B0E042E050E00C944126262F66
:104C2000E199FECF9FBB8EBBE09A01970DB20216B1
:104C300031F02DBB0FB6F894E29AE19A0FBE0895B9
:104C40000396272F0E9410260E940F26252F0E94D0
:104C50001026242F0C9410260196272F0E94102630
:104C60000C940F26262FE199FECF9FBB8EBB2DBB48
:104C70000FB6F894E29AE19A0FBE01960895DC010E
:104C8000CB01FC01E199FECF06C0FFBBEEBBE09A71
:104C900031960DB20D9241505040B8F70895F894F6
:024CA000FFCF44
:104CA200C800BD01010102000500050501191A1B1A
:104CB2001C1D1E1F202122B7221223E422E022DC27
:104CC20022BA22FF5AE200E900EA00B500B600B7B4
:104CD20000CD008301CC008A0192019401210223BC
:104CE2000224022502260227022A02B300B4006F20
:104CF200007000818283E200E900EA00B500B6009C
:104D0200B700CD008301CC008A01920194012102F7
:104D1200230224022502260227022A02B300B4003B
:104D22006F00700081828390919293949596973749
:104D32003635343332076061626364656667000149
:104D4200020202020606060909090909090F0F0FE4
:104D52000F0F0F15151518191919191919191919EC
:044D620019232400ED
:00000001FF
